S123D0007ED0EB7ED1C77ED3484D43465320322E302E320D0A00202320000820080045728A
S123D020726F723A20004E6F7420666F756E6400416C7265616479206578697374004E6F06
S123D040207370616365206C656674004E6F7420656D707479004D697373696E67206F727A
S123D060206D616C666F726D656420617267756D656E74004163636573732064656E6965DB
S123D08064004E6F742065786563757461626C6500536176696E6720004C6F6164696E676F
S123D0A0200053797374656D2074696D65206973206E6F74207365740D0A00436F6D6D611B
S123D0C06E64733A0D0A00466F726D61742059595959204D4D204444204848204D4D20538A
S123D0E0530D0A0073797374656D00BDD74E86F09702CEBC006F00088CBD2A23F8CED009F6
S123D100BDD743BDE38027037ED113BDE0FC26037ED1DEB7BD26CED01EBDD743CEBD26BDFE
S123D120D76EBDD74E7EC0008647BBBC00BBBC01BBBC04BBBC05BBBC06BBBC07BBBC08BB9E
S123D140BC09BBBC0ABBBC0BBBBC0CBBBC0DBBBC0EBBBC0FBBBC10BBBC11BBBC12BBBC13CF
S123D16039B7BD26CED01EBDD743CEBD26BDD76EBDD74E7ED1DE16CED026202416CED03081
S123D180201E16CED056201816CED03E201216CED04C200C16CED074200616CED082200017
S123D1A03CCED01EBDD74338BDD743BDD7588628BD7FE8F7BD26CEBD26BDD76E8629BD7F57
S123D1C0E8BDD74E7ED1DE86F09702BDD128B1BD2B27037ED0EBBDE38027037ED0EBBDE271
S123D1E034CEBC14BDD743CED016BDD743CEBCA06F00BD7FEB81082719810D2727811F23CF
S123D200F1817F22ED8CBD1F27E8BD7FE8A7000820E08CBCA027DB096F003CCED01ABDD7D6
S123D220433820CEBDD74E6F008CBCA027B0FEBC10FFBC94FEBC12FFBC967ED2CBD25CD220
S123D24061D267D26CD274D27BD282D288D291D29AD2A1D2A9D2B0D2BAD2C4006C7300D79A
S123D260E564697200D7E5636400D8786D6B64697200D98D7361766500DA406C6F616400CD
S123D280DB5F72756E00DC0464656C65746500DC2D72656E616D6500DC9B6174747200DD18
S123D2A024746F75636800DD9474696D6500DDDA73657474696D6500DE316D6F6E69746FAC
S123D2C07200DF2F68656C7000DF38CED23DFFBD27CEBCA0FFBD20FEBD276D0026037ED37B
S123D2E002EE00BDD72B270AFEBD270808FFBD2720DF3CCEBCA0FFBD203808EE006E007E1A
S123D300D1DEFEBC0CFFBC94FEBC0EFFBC96CED0E4FFBD20BDE0852702202AA60084C181CD
S123D320C127022020EC01FDBC94EC03FDBC96CEBCA0FFBD20BDE08527022009CCBCA0FDA8
S123D340BD207EE1AF7ED17686F0970286FFA701BDE380270139BDD128B1BD2B270139FFAD
S123D360BD24FCBC10FDBC94FCBC12FDBC96A600810126037ED39F810726037ED3FA8108D4
S123D38026037ED460811026037ED4BF811126037ED539812026037ED5A386FEA70139EC8B
S123D3A002FDBD20EE02EE008C2E002615FEBD2486C1A704FCBC12B3BC10C30001ED056F7B
S123D3C00139BDE085262DFFBD27A600FEBD24A704FEBD27EC03A301C30001FEBD24ED057D
S123D3E0C605FEBD273AA600FEBD243AA7025CC10F23EF4FFEBD24A70139EE04FFBD20BD02
S123D400D77D25037ED45CBDE08526037ED45CFEBD24EE02FFBD20BDE08527037ED45CA69A
S123D42000850226037ED45C3CFEBD24EE04FFBD2038C6103AC61FBDD6724D270A81202729
S123D44006A700085A26F04FA700CEBD2CBDE36C27037ED4564FFEBD24A7013986F120F67C
S123D460EC02FDBD20FDBD22BDE08527037ED4B9A600850226037ED4B985402716BDE0C9E4
S123D48027037ED4B9FEBD22FFBD20BDE08527037ED4B9EC01FDBC98EC03FDBC9A86406F8E
S123D4A000084A26FACEBD2CBDE36C27037ED4B9BDE00F27037ED4B94FFEBD24A70139EC22
S123D4C002FDBD20EC04FDBC9CEE02EE008C2E002617FCBC10FDBC98FCBC12FDBC9AFCBC64
S123D4E09CC31000FDBC9E2027BDE0852645FFBD27A6008501260486F42038EC01FDBC9845
S123D500EC03FDBC9AEC07830001F3BC9CFDBC9EFEBC98FFBC025FCEBD2CBDE35827022046
S123D52012BDE187FEBC02BCBC9A270608FFBC0220E54FFEBD24A70139EC02FDBD20EC0424
S123D540FDBC9CEC06FDBC98EE02EE008C2E002615FCBC98F3BC10FDBC98FEBC98BCBC1220
S123D560232F86F52037BDE0852632FFBD27A6008501260486F42025FCBC98E301FDBC988C
S123D580EC03FDBC9AFEBC98BCBC9A230486F5200CFCBC98FDBC02FEBC9CBDE358FEBD24DB
S123D5A0A70139EC02FDBD20FDBD22EC04FDBC9CEC06FDBC9EFEBD20BDD77D25037ED66C80
S123D5C0BDE085260586F47ED66C8601B7BD26FCBC9EB3BC9C810123088302007CBD26208D
S123D5E0F4B6BD26BDDF6C27037ED66CBDE05727037ED66C3CFEBD24A60884078AA038A76D
S123D60000FCBC98ED01FCBC9AED03FCBC9EB3BC9CC3000124026C06ED07FCBD22FDBD2020
S123D620C6093ABDE278C6073AC61FBDD6724D270A81202706A700085A26F04FA700CEBDE9
S123D6402CBDE36C27037ED66CFEBC98FFBC02BDE15FCEBD2CBDE36C27037ED66CFEBC022F
S123D660BCBC9A270608FFBC0220E44FFEBD24A701393CFEBD20A600270608FFBD20383950
S123D6804F3839BDD672BDD711241848484848B7BD26BDD672BDD7112409BABD26B7BD2618
S123D6A04F0D390C39BDD672BDD711243548484848B7BD27BDD672BDD7112426BABD27B785
S123D6C0BD27BDD672BDD711241848484848B7BD28BDD672BDD7112409BABD28B7BD284F5F
S123D6E00D390C39FEBD20A600270B812F26048620A7000820F1FEBD2039A6002712812014
S123D70027030820F5A6002707812026030820F539271680302B1281092F0C84DF81112BBB
S123D7200881162E0480070D390C39BDD672E6001126064D27030820F21B27058120270139
S123D740394F39A6002706BD7FE80820F639860DBD7FE8860A7E7FE886207E7FE844444433
S123D76044840F8B30813923028B077E7FE8A600BDD75DA600087ED7618DF320F16D00279D
S123D7802DA600272781202723811F2321817E221D8122271981272715812A2711812F27D6
S123D7A00D815C2709816027050820D50D390C39862DE600C54027028664BD7FE8862DE648
S123D7C000C50127028672BD7FE8862DE600C50227028677BD7FE8862DE600C5042702867F
S123D7E078BD7FE839FEBC94BCBC96222BFFBC02CEBD2CBDE35827037ED161CEBD2CA60004
S123D8002708FFBD278D14FEBD27C6403A8CBF2C26ECFEBC020820D07ED1DEBDD7B008BDBC
S123D820D758BDD779BDD758BDD779BDD758BDD779BDD779BDD758BDD779862DBD7FE8BD1C
S123D840D76E862DBD7FE8BDD76EBDD758BDD76E863ABD7FE8BDD76E863ABD7FE8BDD76EEC
S123D860BDD758BDD743FEBD27A60085402705862FBD7FE8BDD74E39FEBD20BDD6FAFFBD50
S123D88020FFBD22A60026037ED1DEA600812E260DA601812E26076D0226037ED937A600B3
S123D8A0812F2621FEBC0CFFBC10FFBC94FEBC0EFFBC12FFBC96862FB7BC144FB7BC15BDD7
S123D8C0D6E47ED878BDD6E4BDE08527037ED176FFBD27A600854026037ED194850126032B
S123D8E07ED194EC01FDBC10FDBC94EC03FDBC12FDBC96CEBC14A60027030820F9FFBD29C1
S123D900FEBD27C6103AFFBD27FEBD27A600271408FFBD27FEBD29A700088CBC932705FFE7
S123D920BD2920E5FEBD29862FA700086F00FEBD22FFBD207ED8788663B7BCA08664B7BC61
S123D940A18620B7BCA2CEBCA3FFBD27CEBC14FFBD29FEBD29A60008FFBD29FEBD27A700D4
S123D96008FFBD278CBD1F26037ED1DE4D26E309096F00A600098CBCA026037ED1DE812F86
S123D98026F16F02CEBCA0FFBD207ED878FEBD20BDD6FAFFBD20FFBD22A60026037ED18265
S123D9A0FEBD22BDD77D25037ED182BDE08526037ED17CBDE05727037ED1888608BDDF6CDB
S123D9C027037ED188BDE05727037ED18886C3A700FCBC98ED01FCBC9AED036F056F06CC28
S123D9E01000ED07FCBD22FDBD20C6093ABDE278C6073AC61FBDD6724D270A81202706A766
S123DA0000085A26F04FA700CEBD2CBDE36C27037ED161CEBD2C6F00088CBF2B23F8FEBC7E
S123DA209AFFBC02CEBD2CBDE36C27037ED161FEBC0209FFBC02BCBC9822E927E77ED1DE16
S123DA40FEBD20BDD6FAFFBD20FFBD22A60026037ED182FEBD22BDD77D25037ED182BDE07C
S123DA608526037ED17CFEBD22BDD6FAFFBD20A60026037ED182BDD6A525037ED182FEBD57
S123DA8027FFBC9CFEBD20BDD6FAFFBD20A60026037ED182BDD6A525037ED182FEBD27FF0E
S123DAA0BC9EBDE05727037ED1888601B7BD26FCBC9EB3BC9C810123088302007CBD2620E0
S123DAC0F4B6BD26BDDF6C27037ED188BDE05727037ED18886A3A700FCBC98ED01FCBC9A57
S123DAE0ED03FCBC9EB3BC9CC3000124026C06ED07FCBD22FDBD20C6093ABDE278C6073AA5
S123DB00C61FBDD6724D270A81202706A700085A26F04FA700CEBD2CBDE36C27037ED16119
S123DB20CED091BDD743CEBC9CBDD779862DBD7FE8CEBC9EBDD779BDD74EFEBC98FFBC02AB
S123DB40BDE15FCEBD2CBDE36C27037ED161FEBC02BCBC9A270608FFBC0220E47ED1DEFE38
S123DB60BD20BDD6FAFFBD20FFBD22A60026037ED182BDD77D25037ED182FEBD22BDD6FA69
S123DB80FFBD20A60026037ED182BDD6A525037ED182FEBD27FFBC9CFEBD22FFBD20BDE045
S123DBA08527037ED176A600850126037ED194EC01FDBC98EC03FDBC9AEC07830001F3BC0F
S123DBC09CFDBC9ECED099BDD743CEBC9CBDD779862DBD7FE8CEBC9EBDD779BDD74EFEBC65
S123DBE098FFBC025FCEBD2CBDE35827037ED161BDE187FEBC02BCBC9A270608FFBC0220DF
S123DC00E47ED1DEFEBC10FFBC94FEBC12FFBC96FEBD20BDD6FAFFBD20FFBD22BDE085274E
S123DC20037ED176FCBD22FDBD207EE1AFFEBD20BDD6FAFFBD20FFBD22A60026037ED18293
S123DC40BDD77D25037ED182BDE08527037ED176A600850226037ED19485402716BDE0C904
S123DC6027037ED18EFEBD22FFBD20BDE08527037ED176EC01FDBC98EC03FDBC9A86406F1A
S123DC8000084A26FACEBD2CBDE36C27037ED161BDE00F27037ED1617ED1DEFEBD20BDD650
S123DCA0FAFFBD20FFBD22A60026037ED182BDD77D25037ED182FEBD22BDD6FAA6002603C9
S123DCC07ED182BDD77D25037ED182FEBD22BDD6FAFFBD20BDE08526037ED17CFEBD22FF2D
S123DCE0BD20BDE08527037ED176A600850226037ED1943CFEBD22BDD6FAFFBD2038C61069
S123DD003AC61FBDD6724D270A81202706A700085A26F04FA700CEBD2CBDE36C27037ED13E
S123DD20617ED1DEFEBD20BDD6FAFFBD20FFBD22A60026037ED182BDD77D25037ED182BDC8
S123DD40E08527037ED176FFBD27FEBD22BDD6FAA60026037ED1825FA600271D84DF8152FF
S123DD60270B8157270B8158270B0820EBCA0120F9CA0220F5CA0420F1FEBD27A60084F89D
S123DD80A700EA00E700CEBD2CBDE36C27037ED1617ED1DEFEBD20BDD6FAFFBD20FFBD221B
S123DDA0A60026037ED182BDD77D25037ED182FEBD22FFBD20BDE08527037ED176A60085C0
S123DDC00226037ED194C6093ABDE278CEBD2CBDE36C27037ED1617ED1DE8647BBBFF8BB4D
S123DDE0BFF9BBBFFABBBFFBBBBFFCBBBFFDBBBFFEB1BFFF27037ED1DECEBD2CBDE278CEB7
S123DE00BD2CBDD779862DBD7FE8BDD76E862DBD7FE8BDD76EBDD758BDD76E863ABD7FE884
S123DE20BDD76E863ABD7FE8BDD76EBDD74E7ED1DEFEBD20BDD6FAFFBD20A60026037EDF77
S123DE4026BDD6A525037EDF26FEBD27FFBD2CFEBD20BDD6FAFFBD20A60026037EDF26BD98
S123DE60D68325037EDF26B6BD26B7BD2EFEBD20BDD6FAFFBD20A60026037EDF26BDD683B3
S123DE8025037EDF26B6BD26B7BD2FFEBD20BDD6FAFFBD20A60026037EDF26BDD6832503C3
S123DEA07EDF26B6BD26B7BD30FEBD20BDD6FAFFBD20A60026037EDF26BDD68325037EDF6D
S123DEC026B6BD26B7BD31FEBD20BDD6FAFFBD20A60026037EDF26BDD68325037EDF26B6CD
S123DEE0BD26B7BD32CEBD2CBDE2FAA601B7BFF9A602B7BFFAA603B7BFFBA604B7BFFCA63B
S123DF0005B7BFFDA606B7BFFE8647BBBFF8BBBFF9BBBFFABBBFFBBBBFFCBBBFFDBBBFFE65
S123DF20B7BFFF7EDDDACED0C7BDD7437ED1DEBDD128B7BD2B7EC000CED0BBBDD7435FCEDA
S123DF40D23DFFBD27FEBD276D00271AEE00BDD758BDD7435CC5032603BDD74EFEBD270871
S123DF6008FFBD2720DFBDD74E7ED1DEB7BD26FEBC04FFBC98FEBC08FFBC02CEBD2CBDE323
S123DF8058270139CEBD2CA6002711FCBC98C30001FDBC98088CBF2C273520EBFCBC98FD97
S123DFA0BC9AA6002611FCBC9AC30001FDBC9A088CBF2C270220EBFCBC9AB3BC984D262121
S123DFC0F1BD26221C271AFCBC9AFDBC9820B8FEBC0208BCBC0A2206FFBC027EDF7B86F2F4
S123DFE039FCBC9A830001FDBC9A09FCBC9AFDBC986C007ABD26270C09FCBC98830001FD39
S123E000BC9820EDCEBD2CBDE36C2701394F39FCBC98FEBC08810123068302000820F6FD92
S123E020BD27FFBC02CEBD2CBDE358270139FCBD27C3BD2C18FCBC9AB3BC986F005D270932
S123E040088CBF2B220E5A20F2CEBD2CBDE36C2701394F3986F239FEBC94BCBC962223FFA5
S123E060BC02CEBD2CBDE358270139CEBD2CA60026024F39C6403A8CBEEC23F2FEBC020872
S123E08020D886F839FEBD20FFBD27FEBC94BCBC962233FFBC02CEBD2CBDE358270139CEC3
S123E0A0BD2CA60027123CC6103AFCBD27FDBD20BDD72B3826024F39C6403A8CBEEC23E26C
S123E0C0FEBC020820C886F939EC01FDBD27EC03FDBC02CEBD2CBDE358270139CEBD2C6D2C
S123E0E0002616088CBF2B23F6FEBC0209FFBC02BCBD2722DE27DC4F3986F5397FBC007F2E
S123E100BC017FBC027FBC03CEBD2CBDE358264CFEBD2C8C4D432644FEBD2E8C4653263CC5
S123E120B6BD3081022635FEBD31FFBC04FEBD33FFBC06FEBD5BFFBC0CFFBC10FEBD5DFF41
S123E140BC0EFFBC12FEBD57FFBC08FEBD59FFBC0A862FB7BC144FB7BC154F3986F139CE5D
S123E160BD2CFFBD27FEBC9CA60008FFBC9CFEBD27A70008FFBD278CBF2C270AFEBC9CBC46
S123E180BC9E220220DF39CEBD2C3A5FFFBD27FEBD27A60008FFBD27FEBC9CA700BCBC9E0C
S123E1A0270C08FFBC9CFEBD278CBF2C26E139A60084A581A527037ED194EC01FDBC98FDF3
S123E1C0BC02EC03FDBC9AEC07830001FDBC9ECEBD2CBDE35827037ED161CEBD2CEC0081C0
S123E1E04727037ED19A5D27037ED19AEC02FDBC9CEC04FDBD29FCBC9EF3BC9C830002FD18
S123E200BC9EC606CEBD2CBDE35827037ED161BDE187FEBC02BCBC9A270608FFBC0220E462
S123E220BDD128B7BD2BFCBD20FEBD293CFEBD20FCBD20398647BBBFF8BBBFF9BBBFFABBBE
S123E240BFFBBBBFFCBBBFFDBBBFFEB1BFFF2621CEBFF8BDE2788647BBBFF8BBBFF9BBBF1D
S11BE260FABBBFFBBBBFFCBBBFFDBBBFFEB7BFFF39CED0A2BDD74339D0
S123E2783637BDE2835D26FA3332395F3CCE9FC0BDE2EC38A10627015CA7063CCE9FC2BD4D
S123E298E2EC38847FA10527015CA7053CCE9FC4BDE2EC38843FA10427015CA7043CCE9F13
S123E2B8C6BDE2EC38843FA10327015CA7033CCE9FC8BDE2EC38841FA10227015CA7023C41
S123E2D8CE9FCABDE2EC38A10127015CA701B6BFF8A7003937A60148484848E600C40F1B3B
S123E2F833398607B79FCF4FB79FCDA600B7BFF8A6013CCE9FCABDE34A38A6023CCE9FC809
S123E318BDE34A38A6033CCE9FC6BDE34A38A6043CCE9FC4BDE34A38A6053CCE9FC2BDE396
S123E3384A38A6063CCE9FC0BDE34A388604B79FCF39371644444444A701C40FE7003339F5
S123E358BDE3A2BDE3BB8601B79FD28620B79FD77EE3D839BDE3A2BDE3BB8601B79FD2863E
S123E37830B79FD77EE3F239BDE387BDE3AC398604B79FD7BDE3A286E0B79FD68601B79F84
S123E398D186EFB79FD7BDE3A239B69FD78480810026F739B69FD7840181002704B69FD1E9
S123E3B8394F39B6BC03B79FD3B6BC02B79FD4B6BC01B79FD5B6BC00840F8AE0B79FD639D2
S123E3D8BDE3A2B69FD784088108260CB69FD0A70008BDE3AC27E9394F39BDE3A2B69FD70D
S117E3F884088108260CA600B79FD008BDE3AC27E9394F39D5
S9030000FC
